:10740000E0E0F0E0859194910196089520E82093C2
:1074100061001092610081E085BF82E085BF81EF4D
:1074200085B987EE84B91DB8769A10BA80EF81BB12
:1074300082E68BB983EF8AB980E58CBD81E08DBD92
:10744000089580EE8BB98BEA57D0109289008AEFAD
:107450008093880082E080936F0083E080938100B6
:10746000E7E0F1E05ED0ED30E9F7A1EEB3E0EDE06A
:10747000F1E003E010E101900D921A95E1F7A059B7
:10748000BF4F0A95B9F756D081E08093D7008AE4C0
:1074900082BF1092D8001092E2001092DA0010928F
:1074A000E10080E808D019BC1EBA1092E00070D448
:1074B00089E05CD481E98093D8000895F201F999BC
:1074C000FECFF2BDE1BD0895F9DFF89A80B508C09E
:1074D000F5DF1FBA80BD0FB6F894FA9AF99A0FBE7D
:1074E00031962F010895A9EAB1E090E81BD08D9361
:1074F0009A95E1F7089586E008D010C083E005D0A2
:107500008F2F10D08E2F0ED080E05E9A59980AC02F
:1075100005D085E0FADF06D080FDFDCF599A5E9850
:10752000089581918EBD8DB5000087FFFCCF8EB58B
:107530000895F4DFE9EAF2E090EB5C98892FF2DF3E
:1075400080E1F0DF5C9AEDDF89EA8E278F77D9F74B
:107550009395983B91F70895E7E9F1E08191908147
:10756000019690838293092E0AF40094009195016C
:1075700006FB5EF00096929111F493959083000CB7
:10758000081620F42E982F982D980895937009F4DA
:107590002E9A913009F42F9A923009F42D9A089579
:1075A000EEE8F1E097819923EAF08FB18095807F32
:1075B000669B88601C9B84609581891310C09681AE
:1075C000992381F49381891306C09481992396E9C4
:1075D00059F080E00AC083839095892304C0858395
:1075E0009AE0968380E09FEF9483828308952E9A99
:1075F0002F9A2D9A22243324EEE8F1E0108611868A
:107600001286E9EAF1E08091900187FD36C084FDA1
:107610004DC082FF089526842220E1F3F894C089AA
:10762000D78520E030E080E090E4AFEFBFEF119627
:1076300082199040E0F72D01B74B8D0127FD13C053
:10764000E6E4F4E011928EE7819392E4E1179193DE
:107650009AE508F092E4E938C9F78193108269DF6E
:10766000FE0121964BDF3FDFF90124D320583F4F25
:10767000040D151D2A9411F7AEC18301282D6090C9
:10768000B2017090B10146D019F48823C1F7089572
:10769000380188243FD0E1F58091B001821709F4C8
:1076A00083016090B4017090B301F4CF6090B40195
:1076B0007090B3012FD081F48823C1F708959FEF14
:1076C00085FD08C086FD05C083FF089599DEE9F3B6
:1076D00082C191E097FB890E6624772483012227DB
:1076E00019D0B1F4882389F38091B00136F088165F
:1076F00050F4821730F0213003C0881520F4281789
:1077000010F48301282F6090B4017090B301E8CF8A
:107710003801822EF301F2DEE6DEC9EAD1E0E0E0D4
:10772000F1E097E009908191081621F49A95D1F73C
:1077300008808010F3CEC9E0D8DECA95E9F7F9DEFB
:0477400088270895F9
:1077440041524455424F59C82F258113AF0000FFC1
:10775400FFCFCFFFFFFFFFCFCFFFFF0000FE067E6E
:107764007E06FE46565616FE0656461EFE3F61E946
:10777400E3FFE3EBE3FFE3EBE3FFE16B3F12011015
:107784000102000008412336000100000000010945
:10779400023E0002010080320904000001020201DD
:1077A4000005240010010424020405240600010736
:1077B4000582030800FF09040100020A0000000713
:0E77C4000504021000010705830210000100F9
:1078000011241FBE8DEF9AE09EBF8DBF04B714BE3A
:1078100088E18093600010926000409100085091D0
:1078200001086F917F91A6C00F928F939F931F9233
:107830000FB60F9211244F936F938091DA0080FF5F
:107840004CC038C00F920FB68F939F93EF93FF9366
:1078500088278093850080938400EEE8F1E097818B
:10786000907261F490818917980B908309F45D9A66
:1078700091818917980B918309F4289A96819150E8
:1078800008F096839481915008F09483881639F417
:107890007C9B05C0B5DD19F0C10101961C01FF916B
:1078A000EF915CC080E189BD82E189BD09B400FE31
:1078B000FDCF08958091D80080FF0FC08091DA003D
:1078C0008E7F8093DA008091D90080FF04C0EADFC8
:1078D00081E08EBB02C019BC1EBA8091E10080FF1E
:1078E0000BC03ED280FF08C03ED28091D80080629B
:1078F000E2DD19BC85E08EBB8091E10084FF1AC0F7
:107900002FD284FF17C0CEDF8091D8008F7DD3DDCA
:107910008FEE2AD025D28F7E816028D28091990166
:10792000882331F48091E30087FD02C081E001C02B
:1079300084E08EBB8091E10083FF0CC011D283FFF5
:1079400009C087EF11D082E08EBB109299010BD055
:107950000AD21ED26F914F910F901F909F918F91DD
:107960000FBE0F9018958EEF0090E1000822009254
:10797000E10008954BDDA0E0B1E0E4E4F7E7059015
:107980000D92AD38E1F71D92BB30E9F701FD0FC054
:1079900000FF03C07C9B0BC008C003FF08C06757F3
:1079A000774729F04757574711F02ADDA1F449DD01
:1079B0002224332431018824ADDE789447D0FDD2CF
:1079C000EFDD7DDE811411F012DEF8CFC5DDC101DF
:1079D000805B964398F3F89489EB8EDD81E0809389
:1079E000E00010926F0010928100109285001092BA
:1079F000840081E085BF15BEC5DD5D9A289A0C9490
:107A00000000A9D107C054D102C0D4D239F0A5D109
:107A100082FFFBCF85FFF7CF8091F1000895082EFC
:107A200083E09AD185FD07C08FD102C0C3D269F02F
:107A300094D180FFFBCF0092F1008091950185FBEE
:107A400026F05D9884E680938E01089584D182FFAC
:107A50004CC18091950185FB26F0289884E680939F
:107A60008F01CFDF182F853431F48CEB94E31C01A8
:107A700025DD8DE008C1843511F4C3DFFACF8C34E5
:107A8000C1F38035B1F3843721F484E4C8DF80E0AA
:107A9000FAC0813611F489E5F6C0813429F4B1DFEA
:107AA000582EAFDF482EE5CF803711F483E5EBC0C9
:107AB000833539F4C0E0D1E08991B1DFC730E1F717
:107AC000E3C0863521F481E3AADF84E3DCC0863796
:107AD00061F481E3669B8E5F1C9B8F5FA0DF8FB19B
:107AE000809582958F708F5BCEC08837A9F489DF2F
:107AF00080939501289A84FD28985D9A83FD5D986E
:107B00002E9881FD2E9A2F9882FD2F9A2D9880FD18
:107B10002D9A87FD8824ADCF8A3649F48FE9F5DCAC
:107B2000C3E000DD7CDFCA95E1F7F8DCADC0833748
:107B300031F487E874DF85E972DF8EE1A4C0853611
:107B400039F4E0E8F3E7C9D0E058F040E0F791CF2E
:107B5000823631F489E563DF80E061DF80E893C03D
:107B6000823419F0873609F07AC02224332449DFA1
:107B7000D82F47DFC82F45DF082F8354843008F003
:107B800081C0063411F4440C551CF20110926F00B0
:107B90001736A1F4033471F483E0B1DCC3DC3FDFBA
:107BA0002197E1F7BBDC08C0063411F4859101C0D0
:107BB0008BDC35DF2197C2F72F0149C00334A1F4D4
:107BC0008E2F8F7021F497DC80E299DCA1DC93DCAE
:107BD00082E095DC16DFA6DCCA95E1F799DC3196E8
:107BE000DA9571F72F0131C00634F1F49F01F437B3
:107BF000D8F473D019C005DF063461F4C0FB46F039
:107C0000F43728F4182E81E087BFE89511243296C6
:107C1000082E0AC0043439F4DF01B370A755BD4FF4
:107C20008D93319601C054DC21972AF7043431F446
:107C30002F01F370FE2B49F47DDC07C0063429F4D4
:107C40002F01F901F43708F446D08DE0E8DE063460
:107C500011F45694479482E080936F0015C08237E8
:107C6000E1E049F08634E0E031F08E34E3E019F0F1
:107C7000813531F4E2E0F0E089E087BF849103C010
:107C80008B3111F08FE3CBDE83E0A4D15DD095FF83
:107C900003C009C08FD149F160D080FFFBCF54D021
:107CA00002C088D111F159D080FFFBCF84E092D17E
:107CB0008BE74BC0A9EAB1E0F437B8F40ED090E4FA
:107CC0000D901D9081E087BFE89532969A95C1F797
:107CD0001124E058F04085E001C083E001D081E14B
:107CE00087BFE89507B600FCFDCF08959091A101EC
:107CF0008091A201913231F0913A61F5813251F5D2
:107D000038D078C0803231F534D054D1E9F08530A4
:107D1000D9F023D083FD18C082FFF7CF04C07CDEEA
:107D20008193615031F09091F3008091F200892BA2
:107D3000B1F7BEDF611549F704C03CD129F08530A9
:107D400019F00BD080FFF9CF8EE79091E8008923DE
:107D50008093E800089584E03DD18091E800089583
:107D60008091E2000895FCDF8E7F80618093E200C5
:107D700008951ED1EAE9F1E067E0089582E061EC40
:107D800009D083E061E802D084E060E842E103C00A
:107D900080E060E042E01ED181E007D01092ED006B
:107DA0006093EC004093ED0008959091EB00892BD7
:107DB0008093EB00089560E0923029F0913031F427
:107DC000EDE362E103C0EFE46EE300C0F1E008958B
:107DD0008091A10188234CF402C0ECD051F0BDDFAA
:107DE00082FFFBCF65CFE6D021F0B7DF80FFFBCF6E
:107DF000ABDF08954091A7015091A80146175105A6
:107E000010F490E028C0611511F0462FFACF9CDFE6
:107E100040E0F7CFCFD059F1853049F19EDF83FDA7
:107E200047CF9BDF82FD20C080FF15C03091F3005B
:107E30002091F20005C081918093F10041502F5FA5
:107E4000411519F028303105B0F350E028303105E4
:107E500009F451E079DF4115E9F65523D9F604C05C
:107E6000A9D029F0853019F078DF82FFF9CF20CF33
:107E7000E1EAF1E0D1DD8193E93AE1F737DF6DDF47
:107E800083FF91C08091A1019091A201913009F1ED
:107E900070F09330F1F0953009F444C0963009F455
:107EA00056C0983009F460C0993059F767C08238DD
:107EB00041F78091A5018DD02091EB001092E9004F
:107EC00077D02295269521702093F1001092F10031
:107ED00052C0882311F08230A1F68F71823089F66A
:107EE0008091A3018823D1F42091A501277049F244
:107EF0002093E9008091EB0080FF10C0933011F4D3
:107F000080E20BC080E151DF81E0880F2A95E9F71C
:107F10008093EA001092EA0088E047DF1092E900BF
:107F200047D02AC0882391F41091A30110680FB79D
:107F3000F8943ED04DDF11DF80FFFDCF1093E300BA
:107F4000103883E009F482E08EBB0FBF2CC080584C
:107F5000823048F58091A3019091A4012CDF60301C
:107F600011F126D047DF1FC08038E9F421D080917D
:107F700099018093F100E8DE2BDF15C0882399F486
:107F80009091A301923078F49093990111D020DF61
:107F900080919901882321F48091E30091E087FD8D
:107FA00094E09EBBEBDED9DE83FF089580E2FDDE28
:107FB00087EFCBCE8EB388230895FCDF69F08091E4
:107FC000E9008F931092E900C8DE83FF01C050DF03
:0A7FD0008F9187708093E9000895F7
:047FFC005DCEFBDC7F
:040000030000740085
:00000001FF
